:0C0000000C9465000C9400000C940000AF
:10000C000C9400000C9400000C9400000C94000064
:10001C000C9400000C9400000C9400000C94000054
:10002C000C9400000C9400000C9400000C94000044
:10003C000C9400000C94C7000C9400000C949400D9
:10004C000C9400000C9400000C9400000C94000024
:10005C000C9400000C9400000C9400001027E80392
:10006C0064000A00010000100001100001000000F3
:10007C000000000000000000000000000000000074
:10008C000000000000000000000000000000000064
:10009C000000000000000000000000000000000054
:1000AC000A0A0A0A0A0A0A0A0A0A0A0A0A0A0A0AA4
:1000BC00010002007A00020004007C000000F894A9
:1000CC00EE27EFBBF1E0F5BFE5BF8DE0A2E0BB276B
:1000DC00ED938A95E9F780E098E0A0E0B1E0ED932C
:1000EC000197E9F7ECEBF0E085919591009761F0C1
:1000FC00A591B59105901590BF01F00105900D9259
:10010C000197E1F7FB01F0CFE8E0EEBBEFEFEDBFBD
:10011C00E8E0EEBFC0E0D3E00C94F502AA93EA93BA
:10012C00FA93EFB7EA931A930A931091C0000091D7
:10013C00C600E12FEC71E9F4E091B603EF5FE093B8
:10014C00B603E150F0E0E356FC4F0083A091B603F8
:10015C00A93119F4E0E0E093B603A091B803AF5FC6
:10016C00A093B803A93129F4E0E0E093B8036894B4
:10017C0024F809911991E991EFBFF991E991A991AD
:10018C0018950A921A926A937A938A939A93AA93DD
:10019C00BA93EA93FA93EFB7EA93E0911F03F091C5
:1001AC0020033196E0931F03F09320030E94C516A1
:1001BC00E1E5F1E00E94C61E0E2E0E94C516E3EA90
:1001CC00F2E00E94C61EE02909F46DC1A091130350
:1001DC00A13029F4F79B02C0F79801C0F79AE1E02F
:1001EC002E26A0916103B0916203809163039091DC
:1001FC0064030E94CA16E0938503F0938603609310
:10020C008703709388030E94D116A9E6B3E00E947D
:10021C00D6160E94DD16A5E9B3E00E94D6160E9400
:10022C00E2160E94EB160E94F71DE0936903F0930F
:10023C006A0360936B0370936C03A0919503B09168
:10024C0096038091970390919803E0E0F0E060E7CB
:10025C0072E40E94F71DE0939503F093960360936C
:10026C009703709398030E94F0160E94F5160E2EB9
:10027C000E94FA160E94F516E02161F1E0919503B7
:10028C00F091960360919703709198030E94E21687
:10029C000E94F71DE0939103F093920360939303F4
:1002AC00709394030E94FF16A3E3B3E00E94081717
:1002BC00A0919103B0919203809193039091940338
:1002CC000E94CA16E0937103F09372036093730358
:1002DC00709374030E940D17E0E0F0E06AE774E499
:1002EC000E9416170E941B170E94591DE093790358
:1002FC00F0937A0360937B0370937C030E94241722
:10030C000E943717A5E4B3E00E943C170E944117E6
:10031C000E940D170E941F1D0E941617E09389035F
:10032C00F0938A0360938B0370938C03A0919903D1
:10033C00B0919A0380919B0390919C030E94591D4C
:10034C00E0939903F0939A0360939B0370939C033F
:10035C00A0911A03E5E20E944A17A7E4B3E00E94B9
:10036C003C170E945A17A0E0B0E080E89FE30E947F
:10037C00F71DA0918903B0918A0380918B03909112
:10038C008C030E94A91DE0938103F0938203609378
:10039C008303709384030E946317A8E1B3E00E9467
:1003AC00E61CEC930E945A170E946C170E94591D70
:1003BC000E947517E0916903F0916A0360916B03D9
:1003CC0070916C030E947E170E943C1E68F5E091B0
:1003DC007103F091720360917303709174030E9426
:1003EC007E170E94591DE0936D03F0936E0360938A
:1003FC006F03709370030E947E170E9487170E94F0
:10040C00521DDF01CB010E94FF160E94F71DA0E0D8
:10041C00B0E081E695E40E94A91DA1E4B3E00E943E
:10042C003C17689423F802C0E8E02E260E945A1765
:10043C00A0917503B0917603809177039091780326
:10044C000E94591DE0937503F09376036093770334
:10045C0070937803A3E2B3E00E940817ABE1B0E01D
:10046C000E94C71F0E949017EA17FB0740F4E09107
:10047C002303F0912403ABE1B0E00E94D71F0E944C
:10048C006C170E94EB160E94A91DA1E2B3E00E941A
:10049C000817A0911103AC3308F4F298A091110342
:1004AC00AC3309F4F29A0E94C516A33AE2E0BE07F7
:1004BC0009F06CC0A0911003E0E00E94C11E0E2E4A
:1004CC000E9495170E949E170E94D81E0E94A31787
:1004DC0091F0E0911103EF5FE0931103E0911003B1
:1004EC00F0E03296A0911103B0E0EA17FB0719F483
:1004FC00ECE3E0931103A0911703A43028F4E091EE
:10050C001703EF5FE0931703E0E0E0931F03E09322
:10051C002003C394A0913703B0913803E8E5F2E0CF
:10052C000E94CC1E0E2E0E94AB17E02199F0E09198
:10053C003703F09138033196E0933703F093380387
:10054C000E9495170E94FA1F2CF4E0E0E093370309
:10055C00E0933803ECE3EC15C9F4CC24E0910003F0
:10056C00EF5FE0930003A0910003AC3379F4E0E07B
:10057C00E0930003E0910103EF5FE0930103A0918E
:10058C000103A43119F4E0E0E0930103E991EFBF1A
:10059C00F991E991B991A99199918991799169917F
:1005AC00199009901895AA93E881E066E0937C0075
:1005BC0085E28A95F1F7E0917A00E064E0937A00A5
:1005CC00E0917A00E071E1F3E0917A00E061E09370
:1005DC007A00E0917800F091790021960895EF97D8
:1005EC0021978EE3A2E0B0E0EEE7F0E00E940F204E
:1005FC00FF2431E050E0E0E8E0936100E0E0E093BC
:10060C006100EFE0E4B9E1E0E5B9E0E0E7B9E8B9B1
:10061C00EAEFEAB9E7EEEBB9E0E0E4BDE3E0E5BD13
:10062C00E0E0E6BDE7BDE8BDE1EAE0938000E2E092
:10063C00E0938100E0E0E0938500E0938400E09398
:10064C008700E0938600E0938900E0938800E093B4
:10065C008B00E0938A00E093B600E1EAE093B000EF
:10066C00E2E0E093B100E0E0E093B200E093B3008D
:10067C00E093B400E1E0E0936E00E0E0E0936F0003
:10068C00E0937000E0936900EDBBE0936800E093A9
:10069C00C000E8E9E093C100E6E0E093C200E0E0CE
:1006AC00E093C500E7E4E093C400E0E8E0BFE0E0DD
:1006BC00E0937F00E0937E00E0E6E0937C00E7E2CD
:1006CC00E0937A00E0E0E0937B00ECBDE093BC00AB
:1006DC0078940E94B0170E94B817EAE09E1650F466
:1006EC00A3E2B0E0E0E0F0E00E94D71FADE1B0E0A3
:1006FC000E94D71F0E94C2170E94C9170E94D017D0
:10070C00E8ECF0E0E0933B03F0933C03ECE0E09387
:10071C000503A0E0B0E00E94CB1FE0930603A1E02C
:10072C00B0E00E94CB1FE0930703A2E0B0E00E9470
:10073C00CB1FE0930803A3E0B0E00E94CB1FE09333
:10074C000A03A4E0B0E00E94CB1FEC8BA5E0B0E064
:10075C000E94CB1FED8BA6E0B0E00E94CB1FEE8B6E
:10076C00A7E0B0E00E94CB1FE0930B03A8E0B0E041
:10077C000E94CB1FE0930C03A9E0B0E00E94CB1FBA
:10078C00E0930D03F798F198AAE0B0E00E94CB1F1C
:10079C00E0931003A9E1B0E00E94C71F0E94D71795
:1007AC00A4E1B0E00E94CB1FE88BA5E1B0E00E9471
:1007BC00CB1FE98BA6E1B0E00E94CB1FEA8BABE02C
:1007CC00B0E00E94CB1FEC87ACE0B0E00E94CB1FE6
:1007DC00ED87ADE0B0E00E94CB1FEE87AFE1B0E05B
:1007EC000E94C71FEB83FC83AEE0B0E00E94CB1FDE
:1007FC00E0931403AFE0B0E00E94CB1FE09316032C
:10080C00A0E1B0E00E94CB1FE0931503ABE1B0E098
:10081C000E94C71FE0932303F0932403A5E7B3E0E2
:10082C000E94D616ADE1B0E00E94C71FA5E6B3E06A
:10083C000E94DC170E948717A1E2B3E00E94081700
:10084C000E946C170E94EB160E94F71D0E947517F0
:10085C00A1E1B0E00E94CB1F2E2FA1E2B0E00E94DC
:10086C00C71FEF83F887A2E1B0E00E94CB1FE88F8F
:10087C00A3E1B0E00E94CB1FEF8BA3E2B0E00E949B
:10088C00C71FA9E7B3E00E94DC17A5E2B0E00E9405
:10089C00C71F0E94E317A7E1B0E00E94CB1FE093B3
:1008AC001A03A8E1B0E00E94CB1F0E940A2022F894
:1008BC00A7E2B0E00E94C71F0E94E817A0910303B3
:1008CC00A43128F4E0910303EF5FE0930303A091BC
:1008DC000303A43189F4E0E0E0931B03E0931C03D1
:1008EC00EBE0E0931D03E8EBE0931E03E0E0E09304
:1008FC00B603EAE0E0930303A091B603AB30A9F48E
:10090C00E091A003E0931B03E091A103E0931C038F
:10091C00E091A203E0931D03E091A303E0931E0377
:10092C00E0E0E093B603E0930303A091B603AC3090
:10093C00C0F0E0E0E0939D03E0939E03E0939F03FF
:10094C00E093A003E093A1030E94C217E0E0E093C0
:10095C00A403E093A503E093A603E093A703E0931D
:10096C00B603E8EC5E1630F45394E4E1E51511F4AB
:10097C00E1E04E2E0E94B017A0E00E94ED173B97CD
:10098C00D8F0A0E00E94F217662777270E94F9178B
:10099C000E944117A8EEB3E080E090E00E94231F74
:1009AC00DF01CB010E940218662777270E94651F82
:1009BC000E94F917E894F3F80E9407180E94B817E0
:1009CC00E7EAE0937A00A2E00E94F217DF01E5E08B
:1009DC00F0E00E94281FBE2E0E940718A3E00E9480
:1009EC00ED178E2E0E940718A7E00E94ED170E2F10
:1009FC000E940718A5E00E94ED171E2F0E940718F1
:100A0C00A0E00E94ED17DE2E0E940718A1E00E94C4
:100A1C00ED17AE2E0E940718A6E00E94ED17EA878C
:100A2C00E7E2E0937A00E1E0E51509F042C0A02F7F
:100A3C00E2E30E94C11E0E2EEAEF0E94BC1EE021D2
:100A4C0011F0E5E0E987A12FE2E30E940E18EAEF2E
:100A5C000E94BC1EE02111F0E6E0E987A02F0E9465
:100A6C001318A02FEEE10E94BC1EE02911F0E7E064
:100A7C00E987A12FEAEF0E940E18EEE10E94BC1E3E
:100A8C00E02911F0E8E0E987EAE08E1620F4EFEFB8
:100A9C008E2EECE00DC0EAE0AE1620F4EFEFAE2E99
:100AAC00EEE006C0EAE0DE1620F4EFEFDE2EEFE01B
:100ABC00E987A02F0E9413180E94181821F0E1E07A
:100ACC00E98708E206C0A02F0E94231811F0E2E08B
:100ADC00E987A12F0E9413180E94181811F0E3E067
:100AEC0005C0A12F0E94231819F0E4E0E9871CE34C
:100AFC00A9850E942818A985E7E00E94A81E0E2A45
:100B0C00E1E00E94A81E0E2AE2E00E94A81EE02945
:100B1C0011F0012F18E2A9850E942D18A985E8E093
:100B2C000E94A81EE02909F018E2A985AE3011F444
:100B3C00EFEFAE2EA985AF3011F4EFEFDE2EA985C5
:100B4C00AC3011F4EFEF8E2E0E9432180E94BC1EB6
:100B5C00E02199F06894F3F8F39B04C0F398F49AAD
:100B6C0032E00BC0F49B04C0F498F59A33E005C056
:100B7C00F59B03C0F598F39A31E0033308F457C0A2
:100B8C000E944118E32F0E944A1808F008EC002E2E
:100B9C001124E32F0E9457180E946818AC91A130C1
:100BAC0008F444C00E946F180E9478180E947F18A5
:100BBC004CF40E9468180E9488180E94681E0E94BB
:100BCC00931829C00E949C180E949E180E94A71876
:100BDC00EF930E949C180E949E180E94AE18AF9131
:100BEC00EA2379F00E9468180E9488180E946D1EF2
:100BFC00A0934903B0934A0380934B0390934C0307
:100C0C000AC00E949C180E949E180E94B5181CF0E5
:100C1C000E94BD180BC0A0914903B0914A0380916A
:100C2C004B0390914C030E9478180E2F03C000E0E8
:100C3C000E94BD180E94C5180E94CB180E220E945B
:100C4C00D018E02129F0009312036894F0F821F8F1
:100C5C00003019F4E89421F810C0A0E021FCA1E0C8
:100C6C00E0E00E94A81E0E2EA09112030E94D7183D
:100C7C0021F0E0E0E093120300E0A0911203A13018
:100C8C0020F0F19A0091120301C0F1980E94DC1837
:100C9C000E94E01E0E94E9180E94F3180E94E81EB0
:100CAC00E02161F10E94F8180E940019A4F0A091B3
:100CBC005503B0915603EB81FC81EA1BFB0BA3E0BF
:100CCC00B0E00E941E1F0E940819AE1BBF0BA09320
:100CDC003D03B0933E030E94F8180E94FA1F2CF4B7
:100CEC000E940D1933970E941219A0913E03AA235A
:100CFC002AF4E0E0E0933D03E0933E030E94DC180D
:100D0C000E94002074F50E94DC180E946D1E0E9447
:100D1C00001974F0AB81BC81E0915503F09156033E
:100D2C00EA1BFB0B0E940819EA0FFB1F0E94121909
:100D3C000E94DC180E946D1EA230E0E0BE07E0E0CD
:100D4C008E07E0E09E072CF00E940D1931960E9450
:100D5C0012190E940819A93CE0E0BE0714F00E9489
:100D6C00C9170E940D19A02FB0E0EA17FB0714F465
:100D7C0000913D030E94171909F008F42DC00E9440
:100D8C002819DF01CB01E0E0F0E060EA70E40E949A
:100D9C003C1E09F008F40CC00E942819A0E0B0E039
:100DAC0080E490E40E94A91D0E9437190E9440190A
:100DBC000E9428190E94F01F34F40E9428190E94E6
:100DCC0037190E944019A0914003AA232AF4E0E0AD
:100DDC00E0933F03E09340030E94171930F50E9403
:100DEC004519DF01CB01E0E0F0E060E470E40E9423
:100DFC003C1E09F008F405C00E9454193A960E9452
:100E0C0040190E9445190E94F01F2CF40E9454199D
:100E1C0033960E944019A0913F03B0914003A13D2D
:100E2C00E7E0BE0714F00E94D017EAE0E09FF00163
:100E3C00DF010E945419EA17FB073CF4A0913F0311
:100E4C00B09140030E9459190E2F0A8F1333A0F052
:100E5C00E0E0E0931203E12FF0E0F2970E949E1E77
:100E6C000E941F1DA6EFB8E28CE99FE30E94A91D0A
:100E7C000E94E61C1E2F01C010E0AB2DE4E60E9480
:100E8C00BC1E0E2EA0E0F099A1E0E1E00E94A81E8D
:100E9C000E94A3171E2E0E945E19A0913703B091D9
:100EAC0038030E94C61E0E9463190E94AB17E021F2
:100EBC00E129B9F0E0912103F0912203ADE1B0E01A
:100ECC000E94D71F0E946B190E94C719A4E6B0E0BC
:100EDC000E94AF1C5F98A8EEB3E00E94AF1C0C946C
:100EEC00B816E0910C03E093B300AA2DEAE00E943F
:100EFC00C11E0E2E0E94CB18E02111F0E894F2F8DE
:100F0C00AA2DE8E60E94241A0E94CB18E02171F069
:100F1C006894F2F8E0911303EF5FE0931303A09150
:100F2C001303A33019F4E0E0E0931303E0911303EF
:100F3C00E03029F4E0E0E093B400F7980FC0A09102
:100F4C001303A13019F4E0910D0306C0A091130313
:100F5C00A23021F4F79AEFEFE093B400A02FE0E079
:100F6C000E940E18E0E00E94C11E0E22A0911303F5
:100F7C000E94D718F9F0E0910403EF5FE0930403AB
:100F8C00A0910403E5E00E94C11E0E2EE4E10E9434
:100F9C00BC1EE02141F0E0910403E170AFEFEA02E6
:100FAC00F001E093B400A0910403A03118F0E0E04C
:100FBC00E0930403EAE0E81510F4E894F1F80E94D9
:100FCC002F1A0E94351A0E94CB18E02131F0689438
:100FDC00F1F85F5F583009F450E00E942F1AA0918D
:100FEC000F03EFEF0E94BC1EE02121F0E0910F03F4
:100FFC00EF5F03C0E894F1F8E0E0E0930F03A091F9
:10100C000F03A431A9F4AA81E0E00E94B71E0E2EB2
:10101C000E94CB18E02119F0EA81E150EA835336A3
:10102C0010F453E605C050E00E946B190E94C719DA
:10103C000E942F1A0E94351AAA81E4E60E94B21E61
:10104C000E943D1A51F06894F1F8EA81EF5FEA834F
:10105C00AA81A43611F4E0E0EA83EAE0E91510F481
:10106C00E894F0F80E94C5180E94D0180E22AA81AC
:10107C00E0E00E94AD1E0E943D1A51F06894F0F819
:10108C00EA81E150EA83AA81AF3F11F4E3E6EA83F7
:10109C00EAE0ED1510F4E894F3F80E9432180E947F
:1010AC00A81EE02109F47EC16894F3F8AA81A1304E
:1010BC0049F4A0910603A13028F4E0910603EF5FF8
:1010CC00E0930603AA81A23049F4A0910703A2334E
:1010DC0028F4E0910703EB5FE0930703AA81A330A8
:1010EC0049F4A0910803A43628F4E0910803EE5FBC
:1010FC00E0930803AA81A43049F4A0910A03A83212
:10110C0028F4E0910A03EF5FE0930A03AA81A5306B
:10111C0031F4AC89A43618F4EC89EF5FEC8BAA811E
:10112C00A63031F4AD89A43618F4ED89EF5FED8B60
:10113C00AA81A73031F4AE89A43618F4EE89EF5F9A
:10114C00EE8BAA81A83049F4A0910B03A13028F4AE
:10115C00E0910B03EF5FE0930B03AA81AD3069F4D0
:10116C00A0912503B0912603A433E8E0BE0728F430
:10117C000E94021831960E94D717AA81AE3031F422
:10118C00A889A43618F4E889EB5FE88BAA81AF3004
:10119C0031F4A989A43618F4E989EB5FE98BAA81AB
:1011AC00A03131F4AA89A43618F4EA89EB5FEA8BF2
:1011BC00AA81A13131F4AC85A83C18F4EC85EB5F25
:1011CC00EC87AA81A23131F4AD85A83C18F4ED85E9
:1011DC00EB5FED87AA81A33131F4AE85A83C18F4FE
:1011EC00EE85EB5FEE87AA81A43169F4A0913503FB
:1011FC00B0913603A835E2E0BE0728F40E945E19D0
:10120C007E960E94E817AA81A53159F4AB81BC8166
:10121C00A33AE1E0BE0728F4EB81FC813196EB8325
:10122C00FC83AA81A63149F4A0911403A53028F4BB
:10123C00E0911403EF5FE0931403AA81A73149F402
:10124C00A0911603A23328F4E0911603EF5FE0930C
:10125C001603AA81A83149F4A0911503A53028F4EE
:10126C00E0911503EF5FE0931503AA81A93119F4FE
:10127C002F3008F42F5FAA81AA3159F40E94441A26
:10128C00AC3BE2E0BE0728F40E94491A31960E945A
:10129C00E317AA81AB3149F4A0911A03AA3F28F4B1
:1012AC00E0911A03EF5FE0931A03AA81AC3161F469
:1012BC00A0E022FCA1E0A13038F4E0E022FCE1E067
:1012CC00EF5F0E940A2022F8AA81AD3169F40E94D6
:1012DC00F016A43FE1E0BE0738F40E94D1163A960E
:1012EC00E0932D03F0932E03AA81AE3169F40E9492
:1012FC00FA16A835E2E0BE0738F40E94DD163A96DD
:10130C00E0933903F0933A03AA81AD3531F4A98DFA
:10131C00A73018F4E98DEF5FE98FAA81AE3561F43F
:10132C00AF81B885A031E7E2BE0730F4EF81F885D4
:10133C00EC59FF4FEF83F887AA81AF3531F4A88DB4
:10134C00A83C18F4E88DE65FE88FAA81A03631F44A
:10135C00AF89A23318F4EF89EF5FEF8BAA81A13626
:10136C0049F4A0911003AC3328F4E0911003EF5F23
:10137C00E0931003AA81A23649F4A0910D03AA3F71
:10138C0028F4E0910D03E65FE0930D03AA81A336E8
:10139C0049F4A0910C03AA3F28F4E0910C03E65FFA
:1013AC00E0930C03EAE0EA1510F4E894F2F8AA2DA5
:1013BC00EAE00E94241AA52FE3E60E94A81EE02171
:1013CC0009F47DC16894F2F8AA81A13049F4A09186
:1013DC000603A13028F0E0910603E150E0930603E8
:1013EC00AA81A23049F4A0910703AB3028F0E09118
:1013FC000703E550E0930703AA81A33049F4A091B9
:10140C000803AD3328F0E0910803E250E0930803A1
:10141C00AA81A43049F4A0910A03A53128F0E091E7
:10142C000A03E150E0930A03AA81A53031F4AC8998
:10143C00A13018F0EC89E150EC8BAA81A63031F484
:10144C00AD89A13018F0ED89E150ED8BAA81A73060
:10145C0031F4AE89A13018F0EE89E150EE8BAA81FF
:10146C00A83049F4A0910B03A13028F0E0910B03B4
:10147C00E150E0930B03AA81AD3069F4A0912503F0
:10148C00B0912603AD36E7E0BE0728F00E940218A3
:10149C0031970E94D717AA81AE3031F4A889A630B3
:1014AC0018F0E889E550E88BAA81AF3031F4A989AE
:1014BC00A63018F0E989E550E98BAA81A03131F406
:1014CC00AA89A63018F0EA89E550EA8BAA81A131E5
:1014DC0031F4AC85A13018F0EC85E550EC87AA818D
:1014EC00A23131F4AD85A13018F0ED85E550ED87D2
:1014FC00AA81A33131F4AE85A13018F0EE85E55008
:10150C00EE87AA81A43161F4A0913503B091360322
:10151C000E94F61F28F40E945E197E970E94E8171D
:10152C00AA81A53159F4AB81BC81A332E1E0BE079D
:10153C0028F0EB81FC813197EB83FC83AA81A631E7
:10154C0049F4A0911403A13028F0E0911403E15068
:10155C00E0931403AA81A73149F4A0911603A23099
:10156C0028F0E0911603E150E0931603AA81A8310C
:10157C0049F4A0911503A13028F0E0911503E15036
:10158C00E0931503AA81A93119F4223008F02150F7
:10159C00AA81AA3159F40E94441AA935E2E0BE0787
:1015AC0028F00E94491A31970E94E317AA81AB31A7
:1015BC0049F4A0911A03A23028F0E0911A03E150EB
:1015CC00E0931A03AA81AC3179F4A0E022FCA1E0EB
:1015DC00A13050F0A0E022FCA1E0E1E00E94C31F8A
:1015EC00EA1B0E940A2022F8AA81AD3161F40E9404
:1015FC00F0160E94F61F38F40E94D1163197E09332
:10160C002D03F0932E03AA81AE3161F40E94FA16D9
:10161C000E94F61F38F40E94DD163197E0933903CF
:10162C00F0933A03AA81AD3531F4A98DA13018F0AD
:10163C00E98DE150E98FAA81AE3559F4AF81B885B7
:10164C000E94F61F30F4EF81F885E456F040EF83EA
:10165C00F887AA81AF3531F4A88DA13018F0E88D48
:10166C00E150E88FAA81A03631F4AF89A13018F08F
:10167C00EF89E150EF8BAA81A13649F4A0911003B8
:10168C00A13028F0E0911003E150E0931003AA81FF
:10169C00A23649F4A0910D03AB3028F0E0910D0374
:1016AC00EA50E0930D03AA81A33649F4A0910C03F0
:1016BC00A13028F0E0910C03EA50E0930C0322FCDB
:1016CC0026C0E0911C03ADE8B3E0FF27662777271F
:1016DC000E941F1D0E94B01FA0918D03B0918E031C
:1016EC0080918F03909190030E94FA1F3CF40E940A
:1016FC004E1A0E94571A0E945E1A09C0E0E0E0934D
:10170C007D03E0937E03E0937F03E093800322FE4E
:10171C000CC0AA85B0E00E945919ADE8B3E00E9454
:10172C00DC170E944E1A0E945E1A0E944E1AA9E102
:10173C00B3E00E94E61CEC93A0911D03B0E0E0E046
:10174C00F1E00E941E1FDF01E0911E03F0E0EA0FA2
:10175C00FB1FADE5B3E00E94DC170E94671AA0E006
:10176C00B0E080E192E40E94F71D7F936F93FF93AA
:10177C00EF930E94441A0E94701AAF91BF918F91FF
:10178C009F91662777270E941F1D0E94A91DE09339
:10179C005D03F0935E0360935F03709360030E949C
:1017AC00751AE0E0F0E060E87FE30E94621E0E2E06
:1017BC000E94751AE0E0F0E068E472E40E945C1E9E
:1017CC00E021F9F00E94671A0E94571AA1E5B3E0D4
:1017DC000E94E81C0E94B01F0E94671AE0936103EC
:1017EC00F093620360936303709364030E94751A11
:1017FC000E94EB160E94A91DA7E2B3E00E940817F5
:10180C0015C0E0E0E0935103E0935203E0935303DF
:10181C00E0935403E0936103E0936203E09363036A
:10182C00E0936403E0932703E0932803A0918103E2
:10183C00B091820380918303909184030E949E1740
:10184C000E94621EEF930E9424170E94621EAF91A9
:10185C00EA2309F43EC0E0911A03F0E0FF93EF9302
:10186C000E941B17E0E0F0E068EC72E40E94F71DA8
:10187C00AF91BF910E94A31E0E94B71F0E94371701
:10188C000E947E1AA0915903B0915A0380915B0378
:10189C0090915C03E0E0F0E064E172E40E94A91D29
:1018AC00DF01CB010E9463170E94F71DA0E0B0E09E
:1018BC0080E291E40E94A91D0E947E1AE0915903D6
:1018CC00F0915A0360915B0370915C03DE010E94FE
:1018DC003C170E94C518A0910E03EDEF0E94BC1E90
:1018EC000E220E94CB18E02129F0E0910E03EF5F4D
:1018FC00E0930E03A92DEAE00E94C11E0E2EA091CA
:10190C000E03EFEF0E94BC1E0E220E94CB18E021AA
:10191C0029F0E894F0F8E0E0E0930E03A0910E03B8
:10192C00EEE10E94A81E0E2E0E94CB18E02119F0A9
:10193C00E1E0E0931103E0911003E03019F4E0E0F2
:10194C00E09311030E9495170E949E170E94E81EB7
:10195C000E946319A09111030E94D71819F0E1E0BD
:10196C00E0931103A0911103AC3309F41FEF442051
:10197C0099F50E94871A0E94E81E0E22A09114036A
:10198C000E94941A1E2E0E94871A0E94E01E0E229C
:10199C00A09115030E94941AE12931F0053108F049
:1019AC000451E0E0E0931703E32FF0E03496DF01FD
:1019BC00EE27A00FBE1FE12F0E94991AA4E00E94EF
:1019CC00BB16A32F0E94A31AA02F0E94BB16A12FF7
:1019DC000E94BB160E94A81AE1E0E41509F057C05A
:1019EC004424A09108030E94B11AE0930903F0E08B
:1019FC00BC96DF01E0910503F0E0AE0FBF1FE09154
:101A0C000603F0E0AE0FBF1FE0910703F0E0AE0F4E
:101A1C00BF1FE0910A03F0E0AE0FBF1FEC89F0E0AE
:101A2C00AE0FBF1FED89F0E0AE0FBF1FEE89F0E0E7
:101A3C00AE0FBF1FE0910B030E94991AACE20E94FB
:101A4C00BB16A09105030E94BB16A09106030E9431
:101A5C00BB16A09107030E94BB16A09109030E941C
:101A6C00BB16A0910A030E94BB16AC890E94BB1640
:101A7C00AD890E94BB16AE890E94BB16A0910B03C8
:101A8C000E94A31AA0E00E94A31A0E94A81A53361F
:101A9C0008F000C3A0E0F799A1E0EA2FE295E07FFF
:101AAC000E2EA0E0F399A1E0EA2FEE0FEE0F0E0E32
:101ABC00A0E0F499A1E0EA2FEE0FA02DAE0FE0E02C
:101ACC00F599E1E0EA0FEB8FEAE0E9ABEAABEBABBF
:101ADC00ECABEDABEEABEFAB0E94B71AEAE0EBAFC1
:101AEC00ECAFEDAFEEAFEFAF0E94BC1AAA34E1E061
:101AFC00BE07E0E08E07E0E09E071CF4E1E0E09317
:101B0C0002030E94BC1AE9E4F1E060E070E00E947C
:101B1C00C51AEEE5F1E060E070E00E94E01EE02105
:101B2C0019F0E3E0E09302030E94BC1AEDE5F1E04A
:101B3C0060E070E00E94C51AE8E6F1E060E070E059
:101B4C000E94E01EE02119F0E7E0E09302030E94FE
:101B5C00BC1AE7E6F1E060E070E00E94C51AECE721
:101B6C00F1E060E070E00E94E01EE02119F0EFE08F
:101B7C00E09302030E94BC1AAC37E1E0BE07E0E040
:101B8C008E07E0E09E071CF0EFE1E09302030E9459
:101B9C009517AA30E0E0BE07E0E08E07E0E09E0774
:101BAC002CF00E9495170E94C81AEBAB0E94951757
:101BBC000E94D11AECABA0911903AA3030F0B0E01E
:101BCC000E9459190E94D51AE9AB0E94DB1AEAABA4
:101BDC000E94E31A0E94ED1A0E94F01AEFAB5030EB
:101BEC0079F5EFEAED8F0E94F31AA436E0E0BE0718
:101BFC0020F00E94F31A0E94F81A0E94F31A0E9415
:101C0C00701A0E94031BEEAF0E94F31A0E94091B6C
:101C1C00A0910103AA3010F0E2E0E8AFA09101031B
:101C2C000E940F1BE9AFA0910003B0E00E9459196C
:101C3C000E94D51AEAAFA09100030E940F1BEBAFD4
:101C4C00513099F5E89420F8EFE4ED8F0E9490174D
:101C5C00A031E7E2BE0728F00E9490170E94151BE6
:101C6C00EBAF0E949017A83EE3E0BE0728F00E945D
:101C7C0090170E941A1BECAF0E949017A436E0E05C
:101C8C00BE0720F00E9490170E94F81A0E9490172D
:101C9C001A9738F00E9490170E94701A0E94031B2A
:101CAC00EEAF0E9490170E94091B523009F069C0D8
:101CBC00E89420F8EFE0ED8FE7E7E9AFE4E7EAAF6F
:101CCC00A0914603AA2352F4E0914503F0914603F8
:101CDC000E94721EE0934503F09346030E94241762
:101CEC000E943717772312F4E0E4EEAF0E9424171A
:101CFC000E9437170E941F1B10F4E0E4EDAF0E9406
:101D0C0024170E9437170E94281B10F4E0E4ECAF54
:101D1C000E9424170E9437170E94311B10F4E0E434
:101D2C00EBAF0E943A1BA031E7E2BE072CF00E94F9
:101D3C003A1B0E943F1BEBAF0E943A1BA83EE3E00C
:101D4C00BE072CF00E943A1B0E94441BECAF0E9471
:101D5C003A1BA436E0E0BE072CF00E943A1B0E940E
:101D6C00491BEDAF0E943A1B1A973CF00E943A1B9C
:101D7C000E9459190E94D51AEEAF0E943A1B0E947C
:101D8C004E1B533009F05BC00E94541BA0914803BA
:101D9C00AA2352F4E0914703F09148030E94721E6B
:101DAC00E0934703F09348030E945D1B772312F4E2
:101DBC00E0E4EEAF0E945D1B0E941F1B10F4E0E4F8
:101DCC00EDAF0E945D1B0E94281B10F4E0E4ECAF09
:101DDC000E945D1B0E94311B10F4E0E4EBAF0E94EB
:101DEC00611BA031E7E2BE072CF00E94611B0E9430
:101DFC003F1BEBAF0E94611BA83EE3E0BE072CF03B
:101E0C000E94611B0E94441BECAF0E94611BA43614
:101E1C00E0E0BE072CF00E94611B0E94491BEDAF55
:101E2C000E94611B1A973CF00E94611B0E94591979
:101E3C000E94D51AEEAF0E94611B0E944E1B5430BB
:101E4C00C9F40E94541BE0E5EBAFA0911803A43633
:101E5C0020F0B0E00E94491BEDAFA0911803B0E058
:101E6C000E9459190E94D51AEEAFA09118030E9436
:101E7C000F1BEFAF553039F5E89420F8EFE8ED8FF4
:101E8C00E0E0E9AFE5E0EAAFE8E7EBAFA881B981C4
:101E9C00A83EE3E0BE071CF00E94441BECAFA881F7
:101EAC00B981A436E0E0BE071CF00E94491BEDAFDF
:101EBC00A881B9810E9459190E94D51AEEAFA88148
:101ECC00B9810E944E1B5630E9F5E89420F8EFE0FA
:101EDC00ED8F1130C0F0ECE0E9AFA12F0E94B11AE8
:101EEC00E436A0E0FA0724F0A12F0E94661BEAAFAB
:101EFC00A12F0E94B11A3A9724F0A12F0E946C1BBB
:101F0C00EBAFA12F17C0EBE0E9AFAA8D0E94B11A7D
:101F1C00E436A0E0FA0724F0AA8D0E94661BEAAF13
:101F2C00AA8D0E94B11A3A9724F0AA8D0E946C1BBC
:101F3C00EBAFAA8DB0E0E2E0F0E00E943B1F0E9404
:101F4C00D51AECAF573009F071C0A0914103B09194
:101F5C004203A135EBEFBE0734F4E1E5FBEFE09370
:101F6C004103F0934203A0914103B0914203A03B83
:101F7C00E4E0BE0734F0EFEAF4E0E0934103F093C1
:101F8C004203A0914203AA234AF4E0E4ECAFE091AF
:101F9C004103F09142030E94721E04C0E091410380
:101FAC00F0914203E0934303F0934403A091430365
:101FBC00B0914403ECE3F0E00E943B1FE0932F034D
:101FCC00F09330030E94721BECE30E94181FA09147
:101FDC004303B0914403AE1BBF0BA0933103B093EA
:101FEC003203EFE2ED8F23FE1BC00E94721B1A9787
:101FFC0010F0E2E0E8AF0E94721B0E94771BE9AF81
:10200C00A0913103B09132030E94701A0E94031BFD
:10201C00EAAFA0913103B09132030E94771BEBAF72
:10202C00E3E7EDAFE8E3EEAFE4E5EFAF0E947C1B36
:10203C00AE2FE0911B030E94821BEA0F0E94881BAB
:10204C000E94911BEC8FA985A130D0F00E94B71A89
:10205C00E9E7EBAFE0E5ECAFEDAFA985B0E00E94AE
:10206C0059190E94D51AEEAFA9850E940F1BEFAF2C
:10207C000E947C1B0E94881BE00DEC8FEFE0ED8F23
:10208C00F29B08C00E947C1B0E94881B0E94911B23
:10209C00EF5FEC8F533609F074C341E0403130F4FC
:1020AC000E949A1BEAE0EC934F5FF8CFAA81ECE513
:1020BC000E94A11BEBE50E94A81EE02911F0EEE1A5
:1020CC00EA83AA81AF3111F4EDE5EA83EA81E030CD
:1020DC0021F4ECE0F0E0ED83FE83AA81A13029F439
:1020EC00E0910603F0E0ED83FE83AA81A23029F48F
:1020FC00E0910703F0E0ED83FE83AA81A33029F47D
:10210C00E0910803F0E0ED83FE83AA81A43029F46A
:10211C00E0910A03F0E0ED83FE83AA81A53021F45F
:10212C00EC89F0E0ED83FE83AA81A63021F4ED89E1
:10213C00F0E0ED83FE83AA81A73021F4EE89F0E074
:10214C00ED83FE83AA81A83029F4E0910B03F0E023
:10215C00ED83FE83AA81A93019F4E0E0ED83EE83D0
:10216C00AA81AA3019F4E0E0ED83EE83AA81AB30AA
:10217C0019F4E0E0ED83EE83AA81AC3021F4E4E2C3
:10218C00F0E0ED83FE83AA81AD3021F40E940218A9
:10219C00ED83FE83AA81AE3021F4E889F0E0ED8373
:1021AC00FE83AA81AF3021F4E989F0E0ED83FE8350
:1021BC00AA81A03121F4EA89F0E0ED83FE83AA81A3
:1021CC00A13121F4EC85F0E0ED83FE83AA81A231EC
:1021DC0021F4ED85F0E0ED83FE83AA81A33121F497
:1021EC00EE85F0E0ED83FE83AA81A43121F40E94F8
:1021FC005E19ED83FE83AA81A53121F4EB81FC816C
:10220C00ED83FE83AA81A63129F4E0911403F0E05A
:10221C00ED83FE83AA81A73129F4E0911603F0E047
:10222C00ED83FE83AA81A83129F4E0911503F0E037
:10223C00ED83FE83AA81A93121F4E22FF0E0ED8336
:10224C00FE83AA81AA3121F40E94491AED83FE83F0
:10225C00AA81AB3129F4E0911A03F0E0ED83FE83FF
:10226C00AA81AC3131F4E0E022FCE1E0F0E0ED8356
:10227C00FE83AA81AD3121F40E94D116ED83FE8339
:10228C00AA81AE3121F40E94DD16ED83FE83AA8172
:10229C00AD3521F4E98DF0E0ED83FE83AA81AE35F6
:1022AC0021F4EF81F885ED83FE83AA81AF3521F40B
:1022BC00E88DF0E0ED83FE83AA81A03621F4EF894E
:1022CC00F0E0ED83FE83AA81A13629F4E09110039E
:1022DC00F0E0ED83FE83AA81A23629F4E0910D0390
:1022EC00F0E0ED83FE83AA81A33629F4E0910C0380
:1022FC00F0E0ED83FE83AA81E0E00E94A11BE3E005
:10230C000E94A61BE1E10E94A61BE2E10E94A61B13
:10231C00E3E10E94A61BE5E10E94A61BEBE10E94F3
:10232C00A61BEDE10E94A81EE02911F0F69A01C04F
:10233C00F698A0E0F699A1E0EA2FE795E0E0E795A2
:10234C00ED8FE0E0EC8FEB8FE0930203AA81B0E01D
:10235C00A7FDBFEF0E9459190E94D51AEBABAA81B9
:10236C00B0E0A7FDBFEFEAE0F0E00E946D1FECAB20
:10237C00AD81BE81A031E7E2BE0718F00E94151BAB
:10238C00EBAFAD81BE81A83EE3E0BE0718F00E9422
:10239C001A1BECAFAD81BE81A436E0E0BE0710F095
:1023AC000E94F81AAD81BE811A9728F00E94AB1BCF
:1023BC000E94031BEEAFAD81BE810E94091BAA8156
:1023CC00E1E10E94A11BE2E10E94A61BE3E10E9455
:1023DC00A61BE5E10E94A61BEDE10E94A81EE029C8
:1023EC0029F00E94AB1B0E94031BEEAFE7EAE093BF
:1023FC007A00A7E00E94ED170E2FE7E2E0937A0037
:10240C00AA810E942818AA81EEE00E94A61BE1E195
:10241C000E94A81EE02911F0E1E06E2EAA810E9414
:10242C002D18AA81EFE00E94A61BE2E10E94A81ED3
:10243C00E02911F0E2E06E2EAA81E7E00E94A11BD8
:10244C00E0E10E94A61B0E94AE1B11F0E3E06E2E91
:10245C00033308F457C00E944118E62D0E944A1815
:10246C0008F008EC002E1124E62D0E9457180E944B
:10247C00B31BAC91A13008F444C00E94BA1B0E945B
:10248C0078180E947F184CF40E94B31B0E94C31B47
:10249C000E94681E0E94CE1B29C00E94D71B0E945E
:1024AC009E180E94A718EF930E94D71B0E949E189B
:1024BC000E94AE18AF91EA2379F00E94B31B0E94E0
:1024CC00C31B0E946D1EA0934D03B0934E038093CB
:1024DC004F03909350030AC00E94D71B0E949E1872
:1024EC000E94B5181CF00E94D91B0BC0A0914D0383
:1024FC00B0914E0380914F03909150030E94781835
:10250C000E2F03C000E00E94D91BAA81AD3049F404
:10251C000E94E31A0E94ED1A0E94F01AEFABE0E25F
:10252C00EB8FAA81A53149F40E94E31A0E94ED1A9F
:10253C000E94F01AEFABE0E6EB8FAA810E942818FC
:10254C00AA81EEE00E94A61BE1E10E94A81EE029F0
:10255C00B1F0A02F0E94B11A0E2FE4E0EB8F0436DD
:10256C0018F00E94E11BEDAB0A3028F00E94E41B2E
:10257C000E94D51AEEABA02F0E940F1BEFABAA81C5
:10258C000E942D18AA81EFE00E94A61BE2E10E9496
:10259C00A81EE029B1F0A02F0E94B11A0E2FE2E084
:1025AC00EB8F043618F00E94E11BEDAB0A3028F0DB
:1025BC000E94E41B0E94D51AEEABA02F0E940F1BA9
:1025CC00EFABAA81E7E00E94A11BE0E10E94A61BF1
:1025DC000E94AE1BB1F0A02F0E94B11A0E2FE1E0A9
:1025EC00EB8F043618F00E94E11BEDAB0A3028F09B
:1025FC000E94E41B0E94D51AEEABA02F0E940F1B69
:10260C00EFABAA81A63121F40E94E71BEBE0ECAF03
:10261C00AA81A73121F40E94E71BE0E4ECAFAA8168
:10262C00A83121F40E94E71BECE0ECAFAA81A931A0
:10263C0069F4A0911903B0E00E9459190E94D51AAF
:10264C00EDAB0E94DB1AEEABE7E7EFABAA81AA3148
:10265C00A9F40E94EE1BE4E6F0E00E94281F0E9401
:10266C00031BEDAB0E94EE1B0E94701A0E94031B11
:10267C00EEAB0E94EE1B0E94771BEFABAA81AB3135
:10268C0059F4ECE7E9AFE7E7EAAFE8E7EBAF0E9414
:10269C00AB1B0E94031BEEAFAA81EDE10E94A11BB4
:1026AC00EEE10E94A81EE029D9F0E3E7E9AFE8E3E8
:1026BC00EAAFAA81AD3111F4EEE501C0E8E7EBAF6A
:1026CC000E94F31B1A9738F00E94F31B0E94701A99
:1026DC000E94031BEEAB0E94F31B0E94771BEFAB17
:1026EC00AA81E1E10E94A11BE2E10E94A61B0E94CB
:1026FC00AE1B11F0E8E7EAAFAA81AD3541F5E7E78B
:10270C00ECAFEEE5EDAFE9E3EEAFE98DEFAFE7EA65
:10271C00E0937A00A98D0E94ED177E2EE7E2E093FC
:10272C007A00E3E6E71528F4A72DB0E00E94491BD8
:10273C00EDABE9E0E71538F4A72DB0E00E9459198C
:10274C000E94D51AEEABA72D0E940F1BEFABAA81EE
:10275C00AE3521F4EEE5E9AFE1E0EAAFAA81AF35A1
:10276C0021F4EEE5E9AFE2E0EAAFAA81A03621F46C
:10277C00EEE5E9AFE3E0EAAFAA81A23611F4E0E1BD
:10278C00EB8F41E0403108F077C00E949A1BEC912E
:10279C00E03021F40E949A1BEFE3EC930E949A1B09
:1027AC00AC91A63021F40E949A1BEDE7EC930E94A9
:1027BC009A1BAC91A13021F40E949A1BE6E0EC9399
:1027CC000E949A1BAC91A23021F40E949A1BEBE55B
:1027DC00EC930E949A1BAC91A33021F40E949A1B9B
:1027EC00EFE4EC930E949A1BAC91A43021F40E946C
:1027FC009A1BE6E6EC930E949A1BAC91A53021F44F
:10280C000E949A1BEDE6EC930E949A1BAC91A730A8
:10281C0021F40E949A1BE7E0EC930E949A1BAC9166
:10282C00A83021F40E949A1BEFE7EC930E949A1BAC
:10283C00AC91A93021F40E949A1BEFE6EC930E9414
:10284C009A1BAC91AA3021F40E949A1BE0E0EC9305
:10285C000E949A1BAC91AB3021F40E949A1BE1E0D0
:10286C00EC930E949A1BAC91AC3021F40E949A1B01
:10287C00E8E0EC934F5F86CFE0910203E695E69596
:10288C000E94F81BEDA90E94FE1BEDA90E94091CD9
:10289C00EDA90E94141CEDA90E941B1CEDA90E941D
:1028AC00221CEDA90E94291CEDA90E94301CEF8F5F
:1028BC00E0910203E695E695E6950E94F81BEEA9D9
:1028CC000E94FE1BEEA90E94091CEEA90E94141C7A
:1028DC00EFA90E941B1CEFA90E94221CEFA90E94C9
:1028EC00291CEFA90E94301CE8A3E0910203E69595
:1028FC000E94F81BEFA90E94FE1BEFA90E94091C65
:10290C00EFA90E94141CEEA90E941B1CEEA90E94A8
:10291C00221CEEA90E94291CEEA90E94301CE9A3DE
:10292C00E8AD0E94F81BE9AD0E94FE1BE9AD0E94C8
:10293C00091CE9AD0E94141CED8D0E941B1CED8D31
:10294C000E94221CED8D0E94291CE0910203E17073
:10295C00EA2BEAA3EDAD0E94F81BEDAD0E94361CEC
:10296C00EDAD0E943F1CEDAD0E94481C0E94521C14
:10297C00EDAD0E94561CEDAD0E945F1CEDADE295D5
:10298C00E170EA2BEBA3ECAD0E94F81BECAD0E94BE
:10299C00361CECAD0E943F1CECAD0E94481CE2952D
:1029AC000E941B1CEEAD0E94561CEEAD0E945F1CDB
:1029BC00EEADE295E170EA2BECA3ED8D0E94681C64
:1029CC00ECAD0E94FE1BECAD0E94091CECAD0E940C
:1029DC00141CEBAD0E941B1CEBAD0E94221CEBAD3A
:1029EC000E94291CEBAD0E94301CEDA3EEAD0E94A1
:1029FC00F81BEEAD0E94361CEEAD0E943F1CEEADF6
:102A0C000E94481C0E946C1C0E941B1CEBAD0E9477
:102A1C00561CEBAD0E945F1CEBADE295E170EA2B0E
:102A2C00EEA3EAAD0E94F81BEAAD0E94361CEAAD9B
:102A3C000E943F1CEAAD0E94481CEE1FE0E0EE1F16
:102A4C000E941B1CEFAD0E94561CEFAD0E945F1C38
:102A5C00EFADE295E170EA2BEFA3EC8DE2950E94CD
:102A6C00F81BEAAD0E94FE1BEAAD0E94091CEAAD00
:102A7C000E94141CE9AD0E941B1CE9AD0E94221C93
:102A8C00E9AD0E94291CE9AD0E94301CE8A7EFAD0E
:102A9C000E94F81BEFAD0E94361CEFAD0E943F1C4C
:102AAC00EFADE695E695E6950E94711CE9A9EE1F3F
:102ABC00E0E0EE1F0E941B1CE9A9E295E170EE0F0D
:102ACC00EE0FEA2BAE2FE9A90E945F1CE9A9E29553
:102ADC00EF70E695E170EA2BE9A7E9A9E695E69592
:102AEC00E6950E94F81BE9A9E695E6950E94771CED
:102AFC00E9A90E947F1CE9A90E94711CEC8D0E941F
:102B0C00521CEC8D0E94821BEA2BAE2FEC8D0E9486
:102B1C00871CEC8DE695E170EA2BEAA7EC8D0E9400
:102B2C00681CEAA9E2950E94771CEAA90E94091C7C
:102B3C00EAA90E948C1CEAA90E94521CEAA90E94D4
:102B4C00821BEA2BAE2FEAA9E6950E94871CEAA904
:102B5C00E170EA2BEBA7EC8D0E946C1C0E94F81B19
:102B6C00EB8D0E94771CEB8D0E947F1CEB8DE69504
:102B7C00E6950E94711CE0910203E2950E941B1CD9
:102B8C00EC8DEE1FE0E0EE1FE170EE0FEE0FEA2B86
:102B9C00AE2FEB8DE695E695E6950E94871CEB8DA6
:102BAC00E295E170EA2BECA7EB8D0E94681CEBA977
:102BBC00E2950E94771CEBA90E94091CEBA90E94CC
:102BCC008C1CECA90E94521CECA90E94821BEA2BC3
:102BDC00AE2FECA9E6950E94871CECA9E170EA2BBC
:102BEC00EDA7EB8D0E946C1C0E94F81BECA9E295E2
:102BFC000E94771CECA90E94091CECA90E948C1C59
:102C0C00EBA90E94521CEBA90E94821BEA2BAE2F4F
:102C1C00EBA9E6950E94871CEBA9E170EA2BEEA7C5
:102C2C000E94901C4D3078F40E94961CA2E5B8E0EE
:102C3C000E94861EE17011F45D9801C05D9A0E949D
:102C4C009D1C4F5FEFCF0E94A51C4D3078F40E9465
:102C5C00961CA0E3B8E00E94861EE17011F45D980A
:102C6C0001C05D9A0E949D1C4F5FEFCF0E94A51C76
:102C7C004D3078F40E94961CA2E0B8E00E94861EAB
:102C8C00E17011F45D9801C05D9A0E949D1C4F5F2C
:102C9C00EFCF0E94A51C4D3078F40E94961CA6E044
:102CAC00B8E00E94861EE17011F45D9801C05D9A37
:102CBC000E949D1C4F5FEFCF0E94A51C4A3098F4D8
:102CCC005E9885E28A95F1F7E9E0E41BA0E4B1E0B7
:102CDC000E94861EE17011F45D9801C05D9A0E94FD
:102CEC009D1C4F5FEBCFE1E0EFA7AFA5A131F8F44E
:102CFC0041E04930C0F45E9885E28A95F1F7EFA582
:102D0C00F0E0DE015E96AE0FBF1FAC91E8E0E41B75
:102D1C000E947E1EE17011F45D9801C05D9A0E94C4
:102D2C009D1C4F5FE6CFEFA5EF5FEFA7DECF5D9A5F
:102D3C0085E28A95F1F7289A8DEC9AE00197F1F7E4
:102D4C00AB2DE4E60E94C11E0E2EA0E0F099A1E08E
:102D5C000E94941A29F0A4E6B0E00E94AF1CF09AED
:102D6C000C946404EF962196FFCFAA93E091C000D7
:102D7C00E072E1F3E881E093C60021960895A091FA
:102D8C001F03B09120030895E0E0F0E061EE75E4DC
:102D9C000E94F71D0895E0912D03F0912E030895E4
:102DAC00662777270E941F1D0E94B01F0895E0918F
:102DBC003903F0913A030895A0916903B0916A0325
:102DCC0080916B0390916C030895E0E0F0E060E279
:102DDC0071E40895A0912D03B0912E030895E0E0C5
:102DEC00F0E00E94D21E0895A0913903B0913A03ED
:102DFC000895E0919103F091920360919303709187
:102E0C00940308950E94E61CED93FC930895A09101
:102E1C007D03B0917E0380917F0390918003089590
:102E2C000E94A91DDF01CB01AFCFA0917903B09116
:102E3C007A0380917B0390917C030895A0911A03EF
:102E4C00E4E6EA9FF001DF01E0917903F0917A0367
:102E5C0060917B0370917C030E94A31E0E94B71F9C
:102E6C0008950E94BA1F0E94521D08950E94E81CEA
:102E7C00ED93FC930895E0915503F0915603609106
:102E8C005703709158030895EA9FF001DF01E09118
:102E9C009903F0919A0360919B0370919C030E949B
:102EAC00A31E0E94B71FDDCFE0918503F09186032E
:102EBC0060918703709188030895E0918103F091EC
:102ECC00820360918303709184030895A09165033C
:102EDC00B091660380916703909168030895E09325
:102EEC006503F0936603609367037093680308951A
:102EFC00A0916D03B0916E0380916F03909170035C
:102F0C000895E0916503F0916603609167037091F9
:102F1C0068030895A0912303B09124030895A09110
:102F2C005103B0915203809153039091540308952F
:102F3C00E0E0F0E060E070E008950E22A091110353
:102F4C00ECE30E94BC1EE0210895A0913503B091E2
:102F5C00360345CFA4E1B0E00E94AF1CE7EAE09352
:102F6C007A000895A4E00E94D902EF2FF0E09E2E83
:102F7C00E7E2E0937A000895EBE0E093A203E8EB3C
:102F8C00E093A3030895E8ECF0E0E0933D03F093A5
:102F9C003E030895E0EDF7E0E0933F03F093400328
:102FAC000895E0932503F093260308950E949E1E36
:102FBC000E941F1D0E94B01F0895E0932B03F093F5
:102FCC002C030895E0933503F093360308950E9483
:102FDC00D902EF2FF0E008950E94D9020E94931EAF
:102FEC000E948F1E0895E0935503F093560360934F
:102FFC005703709358030895E0912503F09126032D
:10300C000895E7E2E0937A00E7EAE0937A00089506
:10301C000E94C11E0E2EA12F0895EAEF0E94C11E20
:10302C000E2E0895A52DE1E00E94C11E0E22A98549
:10303C00E5E00E94BC1EE0210895EEE10E94BC1E5A
:10304C000E2EF0CFE5E00E94A81E0E2E0895E6E0AD
:10305C000E94A81E0E2E0895AD2DEAE00E94BC1E03
:10306C000E2EA0E0F3FCA1E0E0E00E94A81E0E22D0
:10307C00A52FE3E60895E02FF0E0F297ADE7B0E07E
:10308C000E941E1F0F010895F0E0DE011F96AE0F87
:10309C00BF1FEC91F0E0D0010E943B1F0E2F093CAA
:1030AC000895F0E0DE015396AE0FBF1FEC91F0E0F7
:1030BC00D0010E941E1FDF01E4E6F0E00E943B1FDE
:1030CC000E2F0895E32FF0E0DE011B96AE0FBF1F0D
:1030DC000895A0914903B0914A0380914B039091BC
:1030EC004C030895E8EEF3E060E070E00E94651F89
:1030FC000895DF01CB01E02FFF27662777270E9479
:10310C0005200895EC91F0E00E949E1EA8E0BCE41E
:10311C0081E090E00E94651FDCCFE0934903F093BF
:10312C004A0360934B0370934C030895D2DFDACFBC
:10313C00DF01CB01E02FF0E00E949E1E0E946D1E6D
:10314C000895E5E0F0E060E070E00E94E81E08956C
:10315C00E4E1F0E060E070E00E94E01E0895A4312C
:10316C00E0E0BE07E0E08E07E0E09E070895EF8107
:10317C00F885D5DE662777270E94231FCECFA92D91
:10318C00EAE00E94BC1E0E2E0895A52FE3E60E94D5
:10319C00BC1E0895A0E0F0FCA1E0E0E00E94A81E97
:1031AC000895E0E00E94C11EE0210895EB81FC81AE
:1031BC00A0915503B09156038091570390915803F9
:1031CC006627772708950E2EA0915503B0915603CC
:1031DC0080915703909158030895EAE0F0E060E085
:1031EC0070E0089548DEAB81BC81882799270E9446
:1031FC006D1E0895A630E0E0BE07E0E08E07E0E02B
:10320C009E070895A0913D03B0913E030895E0916F
:10321C003D03F0913E030895E0933D03F0933E038C
:10322C000895E22FA0918D03B0918E0380918F03AE
:10323C0090919003FF27662777270E941F1D0E94FD
:10324C003C1E0895E22FF0E0A0918D03B0918E0307
:10325C0080918F03909190030E949E1E0E941F1DCF
:10326C0000CEA0913F03B09140030E94A31E0E9488
:10327C00B71FF7CDE0933F03F09340030895A22FBF
:10328C00BB27E0918D03F0918E0360918F037091B9
:10329C0090030E94A31E0E94B71FE3CDE0913F0351
:1032AC00F09140030895EAE0F0E00E943B1F08957E
:1032BC00E0913503F091360308950E2EA091110381
:1032CC00ECE30E94BC1E0E220895E0910603A0E0E0
:1032DC00B0E00E94DF1FE0910703A1E0B0E00E9484
:1032EC00DF1FE0910803A2E0B0E00E94DF1FE09135
:1032FC000A03A3E0B0E00E94DF1FEC89A4E0B0E079
:10330C000E94DF1FED89A5E0B0E00E94DF1FEE896F
:10331C00A6E0B0E00E94DF1FE0910B03A7E0B0E055
:10332C000E94DF1FE0910C03A8E0B0E00E94DF1FB9
:10333C00E0910D03A9E0B0E00E94DF1FE0911003C3
:10334C00AAE0B0E00E94DF1F57DEA9E1B0E00E94C6
:10335C00D71FE889A4E1B0E00E94DF1FE989A5E14D
:10336C00B0E00E94DF1FEA89A6E1B0E00E94DF1FF7
:10337C00EC85ABE0B0E00E94DF1FED85ACE0B0E087
:10338C0008950E94DF1FEE85ADE0B0E00E94DF1FC4
:10339C00EB81FC81AFE1B0E00E94D71FE0911403F8
:1033AC00AEE0B0E00E94DF1FE0911603AFE0B0E0AA
:1033BC000E94DF1FE0911503A0E1B0E00E94DF1F27
:1033CC00E22FA1E1B0E00E94DF1FEF81F885A1E2BE
:1033DC00B0E00E94D71FE88DA2E1B0E00E94DF1F91
:1033EC00EF89A3E1B0E00E94DF1FE0917903F09137
:1033FC007A0360917B0370917C03A3E2B0E00E949E
:10340C00E81C0E94D71FE0912B03F0912C03A5E23E
:10341C00B0E00E94D71FE0911A03A7E1B0E00E9430
:10342C00DF1FE0E022FCE1E0A8E1B0E00E94DF1F3A
:10343C003FDFA7E2B0E00E94D71F08950E94BC1E98
:10344C000E2EA0E0F2FCA1E0E0E00E94A81E0E22ED
:10345C000895A82DEAE00E94BC1E0E2E0895A0E04F
:10346C00F1FCA1E0E0E00E94A81E0E2208950E22BD
:10347C00A52FE3E60E94A81EE0210895A0912B033E
:10348C00B0912C030895E0912B03F0912C03089537
:10349C00E0918D03F0918E0360918F0370919003F6
:1034AC000895A0E0B0E080E09FE30E94591D0895CC
:1034BC00E0937D03F0937E0360937F03709380030E
:1034CC000895E0915D03F0915E0360915F0370914C
:1034DC0060030895EAE0F0E00E94281F0895A0918F
:1034EC005D03B0915E0380915F039091600308953A
:1034FC00E0935903F0935A0360935B0370935C035E
:10350C000895A0911703E2E00E94C11E0E2EE091D7
:10351C00160305DDFF27662777270895E0E00E9454
:10352C00A81EE0210895F0E0EA0FFB1FE0932903A9
:10353C00F0932A03AEE30C94BB160E94BB16A0E0DA
:10354C000C94BB16E0912A03AE2F0E94BB16A091DF
:10355C0029030C94BB16B0E0E2E0F0E00E943B1FA4
:10356C000895EAE0E8AFE9AFEAAF0895A0915503FA
:10357C00B0915603809157039091580308950E947F
:10358C00E81E21CE2ADE0E94651FDF01CB0125DE5D
:10359C000E947B1F089521DE0E947B1F0895DF018E
:1035AC00EAE0F0E00E946D1F0895A0911903BB277B
:1035BC00EAE0F0E00E946D1F0895D8DFE4E6F0E049
:1035CC0060E070E00E94651FDF01CB01E4CFEDAB42
:1035DC00CDDFD8CFEEABCADFDECFA0912103B09107
:1035EC0022030895E4E6F0E00E94281FDF01EAE0E0
:1035FC00F0E00E946A1FEDAF0895DF01EAE0F0E011
:10360C000E946A1F0895EAE0F0E00E946A1FEFAF83
:10361C000895BB27EAE0F0E00E946D1F0895E0E1F9
:10362C00F7E20E94281FE9CFE8EEF3E00E94281F82
:10363C00E4CFDF01CB01E0E0F0E060E171EC0E944F
:10364C003C1E0895DF01CB01E0E0F0E066EC72EC8B
:10365C000E943C1E0895DF01CB01E0E0F0EC69E72D
:10366C0074EC0E943C1E0895A0914503B091460352
:10367C000895E0E1F7E20E943B1F91CFE8EEF3E002
:10368C000E943B1F8CCFE4E6F0E00E943B1F87CFEB
:10369C00EAE0F0E00E946D1FEFAF0895E89420F887
:1036AC00EFE8ED8FEEE3E9AFE4E7EAAF0895A09120
:1036BC001A03E4E6E9CBA0914703B09148030895BF
:1036CC00B0E0E8ECF0E00E943B1F69CFB0E0E4E131
:1036DC00F0E00E943B1F63CFA0912F03B091300309
:1036EC000895EAE0F0E00E946A1F0895E0911B0340
:1036FC00E170EE0FE0580895E695E695E170EE0F57
:10370C00EE0F08950E2EA0E0F199A1E0EA2FEE0F36
:10371C00EE0FEE0F08950E0EA0E020FCA1E0EA2FB4
:10372C00E295E07FE00D0895E42FF0E0DE01D09605
:10373C00AE0FBF1F08950E94A81E0E2EAA810895D9
:10374C000E94A81E0E2AAA810895AD81BE81C2CE08
:10375C00E3E10E94A81EE0290895E62DF0E0DE01C9
:10376C001B96AE0FBF1F0895A0914D03B0914E0351
:10377C0080914F03909150030895EC91F0E00E94DA
:10378C009E1EA8E0BCE481E090E00E94651FECCF97
:10379C00E0934D03F0934E0360934F0370935003EB
:1037AC000895E2DF9FCCEF81F885B9DB6627772798
:1037BC000E94231FEDCFA02FB0E065CFA02FB0E06B
:1037CC0072CDE9E3E9AFE0E5EAAFEEE3EBAF0895E4
:1037DC00A0912703B09128030895A0913303B091D1
:1037EC0034030895E170E795E0E0E795AE2F089576
:1037FC00E295EF70E695E170E295E07FEE0FEE0F4B
:10380C00EA2BAE2F0895E295EF70E695E695E17000
:10381C00E295E07FEE0FEA2BAE2F0895E295E17072
:10382C00E295E07FEA2BAE2F0895E170EE0FEE0FDC
:10383C00EE0FEA2BAE2F0895E695E170EE0FEE0F2A
:10384C00EA2BAE2F0895E695E695E170EE0FEA2B84
:10385C00AE2F0895E695E695E695E170EA2B08956E
:10386C00E695E170E295E07FEE0FEE0FEA2BAE2FBE
:10387C000895E695E695E170E295E07FEE0FEA2B70
:10388C00AE2F0895E695E695E695E170E295E07F1A
:10389C00EA2BAE2FED8D0895E695E695E695C5CF0E
:1038AC00E295EF70E695E170EE0FEE0FEA2BAE2F7E
:1038BC000895E295EF70E695E695E170EE0FEA2B30
:1038CC00AE2F0895E295EF70E6958CCFE295EF70F0
:1038DC00E695E6950895E170E295E07FEA2BAE2F30
:1038EC000895E170E295E07FEE0FEE0FEA2BAE2F1C
:1038FC000895E695E170E295E07FEE0FEA2BAE2F8E
:10390C000895E170EE0FEA2BAE2F0895E295EF705B
:10391C00E695E1CF289885E28A95F1F741E0089584
:10392C005E9885E28A95F1F7ECE0E41B089585E258
:10393C008A95F1F75E9A85E28A95F1F708955D9A7A
:10394C0085E28A95F1F7289A84E191E00197F1F7E5
:10395C00E1CF109639F08DEC9AE00197F1F7A8952C
:10396C001197C9F70895552342F4503811F4E0FF2C
:10397C0004C03196691F791F6BF050E8572711F47A
:10398C005F93CFC05F3F31F0660F000C5795679582
:10399C00752F08955F9300200AF0CFC0C8C050E87F
:1039AC00192E1522880F991F9527550F879550E8CA
:1039BC00072E0522660F771F7527550F67950895FB
:1039CC00689401C0E8945F93F2DF703818F07F3F81
:1039DC0008F4A7C056E1571BAAF4519558300EF4C1
:1039EC00593030F0EFEFFFEF6FEF7FE777F91AC048
:1039FC0077275523B9F0EE0FFF1F661F771F5A95D7
:103A0C00D1F710C07727583028F0EF2FF62F672FFB
:103A1C005850F9CF552331F076956795F795E79582
:103A2C005A95D1F700200AF45BD15F910895689400
:103A3C0001C0E894309760407040B1F0002426F04B
:103A4C00772312F400944CD1172E7EE1112032F022
:103A5C007A95EE0FFF1F661F111CF9CFEF2FF62F73
:103A6C00612D5F938ADF5F9108954F93AF01FD0144
:103A7C00DA01AB01BC01CA01402D012C142E4F916F
:103A8C000895EA0FFB1F681F0895E095F095609567
:103A9C00EF5FFF4F6F4F08955F9381DF903871F1A7
:103AAC0050E8152604C05F937ADF903839F17038EE
:103ABC0021F1572F591B2BF112F4D7DFFACF5831C4
:103ACC0018F0AA27BB278827583028F0AB2FB82F1F
:103ADC0088275850F9CF552329F08695B795A79587
:103AEC005A95D9F7502D512572F0CBDF38F46795E4
:103AFC00F795E795739513F420C0B7DF3EDF5F9120
:103B0C000895D8F7FBCFEA1BFB0B680B51F010F4B0
:103B1C000094BBDF662392F3EE0FFF1F661F7A95AE
:103B2C00CBF7EE27FF27662777275F910895EFEFF6
:103B3C00FFEF6FE77FEF5F910895EFEFFFEF6FE718
:103B4C007FE75F9108955F932ADF703851F39038C7
:103B5C0041F301240894791F23F41CF300203AF359
:103B6C00ECCF0F921F932F933F934F931127222744
:103B7C009927689FA0018F9F302D410D591F6B9F76
:103B8C00300D411D591F8E9F27D0BF9F25D06A9F96
:103B9C0023D0BE9F1DD0AF9F1BD0AE9F110D291FF0
:103BAC00391F491F591FE32FF42F652F522F4F91A7
:103BBC003F912F911F910F9066232AF0550FEE1F06
:103BCC00FF1F661F02C073954BF2CDDE5F91089507
:103BDC00100D211D391F02C0200D311D491F591F09
:103BEC0008955F93DCDE703821F411200AF49FCF26
:103BFC00A4CF903809F495CF01240894970B1BF4AB
:103C0C00D4F30020F3CF792F1F932F933F934F932F
:103C1C0011241127222733274427552790E2AE176A
:103C2C00BF078607410730F0AE1BBF0B860B410B5D
:103C3C00089401C08894551F221F331F111CAA1F02
:103C4C00BB1F881F441F9A9551F7F901612D4F91A5
:103C5C003F912F911F91662332F0550FEE1FFF1FDE
:103C6C00661F7A9543F27FDE5F91089599239AF04F
:103C7C00772342F0971748F029F4AE17BF07860751
:103C8C0020F031F0989488940895989408940895AD
:103C9C001894889408957723C2F7971798F3A9F787
:103CAC00EA17FB07680788F399F3ECCFDFDFE1E055
:103CBC0009F008F0EE270895D9DFE1E009F008F4E7
:103CCC00EE270895EA0FFB1F681F791F0895AE1B9E
:103CDC00BF0B860B970B0895F195E195F040089575
:103CEC00F09560957095E195FF4F6F4F7F4F08955C
:103CFC00EE230E2EEA2F19F0E6950A94E9F70895B3
:103D0C00EE230E2EFD0121F0F695E7950A94E1F7CE
:103D1C000895F695E795F695E795F695E795F6955A
:103D2C00E7950895FE2FFF0FFF0B6F2F7F2F089540
:103D3C006F2F660F660B762F08958B2F880F880BCD
:103D4C00982F0895EA17E1E009F0EE270895AE17D1
:103D5C00E1E00CF4EE270895AE17E1E00CF0EE274D
:103D6C000895EA17E1E00CF0EE270895AE17E1E0B4
:103D7C0008F0EE270895EA17E1E008F0EE27089521
:103D8C00EA17FB07E1E009F0EE270895AE17BF072D
:103D9C00E1E008F0EE270895EA17FB07E1E008F0F0
:103DAC00EE270895EA17FB0768077907E1E009F0A9
:103DBC00EE270895AE17BF0786079707E1E00CF0D2
:103DCC00EE270895EA17FB0768077907E1E00CF086
:103DDC00EE270895FA9FF02DEB9FF00DEA9FE02D52
:103DEC00F10D08957A9F702D6B9F700DF89F700DDB
:103DFC00E99F700D6A9F602D710DFB9F600D711D09
:103E0C00E89F600D711D8827FA9FF02D610D781FBA
:103E1C00EB9FF00D611D781FEA9FE02DF10D681FDF
:103E2C00781F08956E2F6A9FF0016B9FF00D089517
:103E3C0070D0D0DF0EF450DF089579D0D3DF0EF4BC
:103E4C004FDF08950024112490E1AA0FBB1F001C22
:103E5C00111C0E1A1F0A18F40E0E1F1E01C0A160B1
:103E6C009A9599F7FD01D001089553D0EBDF0EF42C
:103E7C0033DF08953F934F935F930024112444271D
:103E8C00552730E2AA0FBB1F881F991F001C111C5D
:103E9C00441F551F0E1A1F0A460B570B28F40E0E03
:103EAC001F1E461F571F01C0A1603A9559F7FD010F
:103EBC00BC01D001CA015F914F913F91089537D059
:103ECC00D9DF0EF40DDF0895BDDFFD010895E894F0
:103EDC00B7FF04C0A095B09511966894F7FDFCDE71
:103EEC00B1DFFD010EF4F8DE0895E89497FF09C0E8
:103EFC00A095B09580959095AF5FBF4F8F4F9F4F1A
:103F0C00689477FDEDDEB6DFFD01BC010EF4E8DE52
:103F1C000895E894F7FF02C0DFDE6894B7FF06C08F
:103F2C00A095B095119600F8039400FA0895E894C2
:103F3C0077FF02C0D5DE689497FF0BC00024A095D4
:103F4C00B095809590951196801D901D00F8039466
:103F5C0000FA0895ED93FD936D937C930895689406
:103F6C0001C0E89401D066DD182E862F612D192E24
:103F7C00972F712D1B2EBF2FF12D1A2EAE2FE12D49
:103F8C000895119602D0FE2F1197F999FECFFF9349
:103F9C00FFB7F894A1BDB2BDF89AE0B5FFBFFF9191
:103FAC00089507D01196EF93EF2F03D0EF9111974F
:103FBC000895F99B02C0A895FCCF9FB7F894A1BDBA
:103FCC00B2BDF89A80B5E81719F0E0BDFA9AF99AE3
:103FDC009FBF089500240E160F06060607060895C7
:103FEC0000240A160B06089500240A160B06080670
:103FFC0009060895EA17FB07680779070895AE17B5
:10400C00BF07860797070895E894EE2309F0689494
:10401C000895AC0FBD1F05900D928A95E1F7089598
:00000001FF
